:100000000C9437050C9498050C9440080C949805B2
:100010000C9498050C9498050C9498050C949805EC
:100020000C9498050C9498050C9498050C94E7147E
:100030000C9498050C94AC220C9498050C9498059B
:100040000C9498050C9498050C9498050C941C231A
:100050000C9498050C9498050C9498050C949805AC
:100060000C9498050C9498050C9498050C9498059C
:100070000C949805BF09C109CD09CD09CD09CD0959
:10008000CD09CD09C309C509C709CD09CD09C109E4
:10009000CF09CD09CD098909BF09CD09CD09C50908
:1000A000CD09CD09CD09CD09CD09CD09C709BF09B4
:1000B000AB09CD09AF09CD09CD09CD098B09C3091C
:1000C000CD09CD09B909CD09CD09CD098D09CB09D6
:1000D000CD09AD09CD09C109CD09CD09BD09B109C8
:1000E000CD09B309C509CD09CD09CD09BB09B509AC
:1000F000CD09CD09CD09CD09CD09CD09CD09B70966
:10010000CD098F09CD09CD09C309CD09CD09CB0989
:10011000CD09CD09CD09CD09CD09CD09CD09CD092F
:10012000CD099109CD09CD09CD09B909CD09CD096F
:10013000CD09CD09CD09CD09CD09CD09CD09CD090F
:100140009309CD0995099709CD09CD09CD099909DB
:100150009B099D09CD099F09A109CD09CD09CD09AB
:10016000C909A309CD09A709A509A909CD09CD097F
:10017000CD09CD09CB09F309010A0D0A0D0AE509DC
:100180000D0A0D0A0D0A0D0A0D0A0D0A0D0A0D0AB7
:100190000D0A0D0A0D0A0D0A0D0AE7090D0AE909F3
:1001A0000D0A0D0A0D0A0D0A050A0D0A1C0A030A9A
:1001B0000D0A0D0A0D0A0D0A0D0A0D0A0D0A0D0A87
:1001C0000D0A0D0A0D0A0D0A0D0ADD09F909EB09E0
:1001D000FD090D0AED090D0AF1090D0AFB09EF09E8
:1001E000FF09F509F7090D0A0D0A0D0A0D0A0D0A96
:1001F0000D0A0D0ADF09E109E309070A090A0D0AD8
:100200000D0A0D0A0B0A9A0AB00ABE0ACC0AEC0AB9
:10021000030B260B430BCB0BF80B8F0CEA0CD00C0B
:10022000FF0C140D1E0D250D290D300D4D137413EB
:100230006C1474136C14C013E3136C143A14491443
:1002400089188918B318B3180E19391B391B391BB3
:100250004219391B2D1A2D1AF31A391B081B261B9C
:10026000807B01484746293A687F0277762B353BE9
:100270006978796439141E3C6A7A1D16041A1F3D88
:100280006B061B070821203E6C2C19091715223F0D
:100290006D11050B0A1C23406E7E100D182425419C
:1002A0006F360E0C122726427037380F33132D434A
:1002B000717534322F2E44727C7D28303174457331
:1002C000515065524C4D2A4900594F5C5F4E4A4B84
:1002D00062635A5D5E60535467585B66576155565A
:1002E0004842403E3C3A3B456843413F3D2B357ECA
:1002F000697A790078141E7C6A7B1D16041A1F7FA8
:100300006B061B070821204D6C2C19091715224A72
:100310006D11050B0A1C234C6E49100D1824255134
:100320006F360E0C1227264F7037380F33132D52AD
:10033000717534502F2E4E72397D283065314B73D4
:100340005464586776012A773259745C5F660246B6
:1003500062635A5D5E60295344575B56556147039B
:1003600080291E1F20212223242526272D2E2A2BDB
:10037000141A0815171C180C12132F30287804169D
:1003800007090A0B0D0E0F33343579311D1B061981
:100390000511103637387D557A2C393A3B3C3D3EB5
:1003A0003F4041424353475F6061565C5D5E575931
:1003B0005A5B62634648324445677B7F65030102AE
:1003C0005250514F68696A6B6C6D6E6F70717258E4
:1003D00000494C754A4D734B4E767C777E7466545B
:1003E000722530325820006225303458200077259D
:1003F0003032582000214353335F4630210A002118
:100400004353335F46305F455252210A0021435324
:10041000335F46305F4F5652210A00214353335F0A
:100420005245414459210A00214353335F455252FA
:10043000210A00214353335F4F5652210A002143C2
:1004400053325F45305F4630210A00214353325F0B
:100450004630210A00214353325F4530210A0021F2
:100460004353325F494E4954210A00214353325FBE
:10047000455252210A00214353325F4F5652210AFE
:1004800000214353315F45305F25303258210A0047
:10049000214353315F455252210A00214353315FBA
:1004A000494E56210A004C25752000532575200021
:1004B00049443A25303458282564290A004D6F757F
:1004C00073653A206E6F7420737570706F72746507
:1004D000640A000A4552523A253032580A00522521
:1004E0007520005725752000572575200057257564
:1004F000200058257520004925752000696E697413
:100500000A000A4552523A253032580A000A4B6511
:1005100079626F6172642073746172742E0A000ACA
:1005200055534220636F6E666967757265642E0A63
:10053000000A0A544D4B3A66396662393737302F14
:100540004C5546410A0A003403490042004D002040
:10055000005000430020006B006500790062006FCE
:1005600000610072006400200063006F006E00767E
:10057000006500720074006500720000000E0374D4
:10058000002E006D002E006B002E000000040309F9
:100590000409027400040100A032090400000103F0
:1005A000010100092111010001224000070581031A
:1005B00008000A09040100010300000009211101DB
:1005C00000012236000705820308000A0904020020
:1005D0000203000000092111010001222200070589
:1005E0008303200001070503032000010904030021
:1005F0000103000000092111010001223900070553
:1006000084032000011201100100000008EDFEEE3D
:100610001B01000102000105010906A101050719DE
:10062000E029E715002501950875018102050819E3
:100630000129059505750191029501750391010543
:1006400007190029F71500250195F875018102C0E9
:100650000631FF0974A1010975150026FF009520D8
:10066000750881020976150026FF0095207508910E
:1006700002C005010980A10185021601002637008C
:100680001A81002AB700751095018100C0050C0978
:1006900001A1018503160100269C021A01002A9C73
:1006A00002751095018100C005010906A101050729
:1006B00019E029E7150025019508750181029501CA
:1006C0007508810105081901290595057501910233
:1006D0009501750391010507190029FF150026FFF3
:1006E00000950675088100C0636F6E73756D657245
:1006F0003A20253034580A0073797374656D3A20B6
:10070000253034580A000A002530325820006B6525
:1007100079626F6172643A20004C45443A2025307A
:1007200032580A00253032583A2025303862257375
:100730000A00722F632030313233343536370A00E5
:1007400064656C5F6B65795F6269743A2063616EA2
:1007500027742064656C3A20253032580A006164A1
:10076000645F6B65795F6269743A2063616E2774B8
:10077000206164643A20253032580A003F00433E2D
:1007800020004C25640A000A092D20436F6E736F08
:100790006C65202D0A4553432F713A0971756974B0
:1007A0000A000A092D204D61676963202D0A643A09
:1007B0000964656275670A783A096465627567203D
:1007C0006D61747269780A6B3A09646562756720B5
:1007D0006B6579626F6172640A6D3A09646562756E
:1007E00067206D6F7573650A763A0976657273696D
:1007F0006F6E0A733A097374617475730A633A0908
:10080000636F6E736F6C65206D6F64650A302D3495
:100810003A096C61796572302D34284631302D46A5
:1008200034290A506175733A09626F6F746C6F6195
:100830006465720A6E3A094E4B524F0A003F004EF1
:100840004B524F3A206F66660A004E4B524F3A2089
:100850006F6E0A0074696D65725F72656164333230
:1008600028293A202530346C580A006B6579626F6C
:100870006172645F6E6B726F3A2025580A006B6577
:1008800079626F6172645F69646C653A2025580A09
:10089000006B6579626F6172645F70726F746F6311
:1008A0006F6C3A2025580A00686F73745F6B657926
:1008B000626F6172645F6C65647328293A20255801
:1008C0000A000A092D20537461747573202D0A00E3
:1008D0004743433A20352E342E30204156522D4C7A
:1008E0004942433A20322E302E30204156525F4149
:1008F0005243483A2061767233350A004F505449CA
:100900004F4E533A204C5546412045585452414B86
:10091000455920434F4E534F4C4520434F4D4D4179
:100920004E44204E4B524F204B45594D41505F5342
:10093000454354494F4E20424F4F544C4F4144453C
:10094000525F53495A450A004255494C443A206681
:1009500039666239373730202831343A33303A310A
:1009600036204D61722020322032303230290A0088
:100970005649443A2030784645454428742E6D2E19
:100980006B2E29205049443A203078316265652821
:1009900049424D205043206B6579626F617264203B
:1009A000636F6E76657274657229205645523A20DF
:1009B0003078303030310A00444553433A20636F79
:1009C0006E766572742049424D205043206B6579E4
:1009D000626F61726420746F205553420A000A09E5
:1009E0002D2056657273696F6E202D0A000A6D6F97
:1009F0007573653A206F66660A000A6D6F757365D8
:100A00003A206F6E0A000A6B6579626F6172643A10
:100A1000206F66660A000A6B6579626F6172643ADC
:100A2000206F6E0A000A6D61747269783A206F66F1
:100A3000660A000A6D61747269783A206F6E0A0066
:100A40000A64656275673A206F6E0A000A6465621F
:100A500075673A206F66660A000A0A626F6F746CE7
:100A60006F616465722E2E2E2000433E20001124FB
:100A70001FBECFEFD4E0DEBFCDBF04B603FE41C042
:100A80008091850390918603A0918703B09188039C
:100A90008730904BA740B04BA1F510928503109280
:100AA0008603109287031092880314BE0FB6F89441
:100AB000A89580916000886180936000109260002A
:100AC0000FBE1092010810920008E3E0F0E089E008
:100AD00080935700E491E695E370E150E33040F4F1
:100AE000F0E0EE0FFF1FE35DFE4F8081918102C0B9
:100AF00080E090E1E0E0F0E8E81BF90BF695E7957F
:100B0000099511E0A0E0B1E0E2E6FAE402C0059048
:100B10000D92A433B107D9F723E0A4E3B1E001C0FB
:100B20001D92A538B207E1F70E9467100C942F259B
:100B30000C940000FF93EF93E0913401F0913501A4
:100B4000309709F00995EF91FF910895FC01859187
:100B5000803011F0EFDFFBCF0895FF27E0E230E2B5
:100B600047FF0CC0419597FF09C0EDE26095709575
:100B700080959095611D711D811D911D27FF02C0FB
:100B8000219530E350E2AA27660F771F881F991F2F
:100B9000AA1FA41710F0A41B63955A95A9F7AA30B1
:100BA00008F0A95FA05DAF93F3956115710581050C
:100BB000910541F7ED3211F4EF93F395F21718F424
:100BC0003F93F395FBCF8F91B5DFFA95E1F7089549
:100BD000E991F9918591803021F0853219F0AADFF1
:100BE000F9CF089520E0E89455915532C1F3503380
:100BF00011F4689455915A3348F4505390F3220FEE
:100C0000022E220F220F200D250FF4CF0EF4219576
:100C100089919991533619F3533729F1533559F185
:100C2000BC0188279927E8945C3621F48991999131
:100C300068945591543639F446EF7EF077FF0DC035
:100C40008FEF9FEF0AC055374AE039F0583540E141
:100C500021F0523642E009F00895FF93EF937DDFD3
:100C6000EF91FF91B7CFFF93EF93FC01819180301B
:100C7000B9F360DFFBCFFF93EF9368DFF1CFDF9332
:100C8000CF93CDB7DEB72596A3DFCF91DF9108953F
:100C900090913F01923081F09330D1F0913031F555
:100CA000E72FF0E0B3E0EE0FFF1FBA95E1F7E60F94
:100CB000F11DE05AFC4F17C0E72FF0E0A3E0EE0F64
:100CC000FF1FAA95E1F7E60FF11DE052FD4F0BC0A3
:100CD000E72FF0E073E0EE0FFF1F7A95E1F7E60FE4
:100CE000F11DE05AFD4FE491E03819F480E090E006
:100CF000089590E023E0880F991F2A95E1F72E2FA1
:100D0000207730E044E0359527954A95E1F7820F4A
:100D1000931F54E0880F991F5A95E1F7EF709C01DB
:100D20002E0F311DF901EE0FFF1FE050F84985919C
:100D3000949108955998519A08955198599A0895FF
:100D40005898509A08955098589A08955198599AD9
:100D500085E08A95F1F7000089B186958170089544
:100D60005098589A85E08A95F1F7000089B1817012
:100D70000895CF93DF93EC010E94A606882341F0EB
:100D8000209731F085E08A95F1F700002197F4CFA4
:100D9000CE01DF91CF910895CF93DF93C2E3D0E0EE
:100DA0000E94A606811108C0209731F085E08A953F
:100DB000F1F700002197F4CFCE01DF91CF91089594
:100DC0002E9826982F9827980E949A060E94A3068C
:100DD000E9E6F0E0808188608083E9980895E19AEF
:100DE000E99A0E949D060C94A306E9980E949A062F
:100DF0000C94A306CF932FB7F894809102019091A1
:100E00000301AC01442741155F4F21F0C92FAC010C
:100E10005F6F07C08F3F4FEF940741F0C82F4FEF30
:100E20005FEF509303014093020101C0CFEF2FBF4A
:100E30009C012F6F2F3F3F4F81F02091720320FFC5
:100E40001FC09F938F9387EE93E09F938F930E9491
:100E50003F060F900F900F900F90CF3F99F0809129
:100E6000720380FF12C01F92CF9380EE93E09F9396
:100E70008F930E943F060F900F900F900F9005C028
:100E8000CF3F19F48FEF9FEF02C08C2F90E0CF91EE
:100E90000895CF93CAE1C15069F00E94FA068F3FCE
:100EA0002FEF920749F48FE99FE00197F1F700C017
:100EB0000000F1CF8FEF9FEFCF91089580E090E891
:100EC00090930101809300018FEF9FEF90930301B6
:100ED000809302010895EF92FF920F931F93CF9397
:100EE000DF93082F109237018091720380FF0CC0AE
:100EF0001F920F938EEE93E09F938F930E943F0675
:100F00000F900F900F900F90E9980E949A060E9400
:100F1000A3068FE891E00197F1F700C000000E945E
:100F2000A0060E949D0680E197E20E94B906892BE7
:100F300011F481E079C0C0E0D0E0FF24F39410E028
:100F4000EE24E39490E59A95F1F7C8010C2E02C0C7
:100F5000959587950A94E2F780FF04C0FE240E94CD
:100F6000A30602C00E94A0060E94CC06892B11F4A1
:100F700082E05AC082E390E00E94B906892B11F406
:100F800083E052C02196C830D105E1F680E58A950C
:100F9000F1F7FF2019F00E94A30602C00E94A006EC
:100FA0000E94CC06892B11F484E03EC082E390E0DD
:100FB0000E94B906892B11F485E036C090E59A9518
:100FC000F1F70E94A306C2E3D0E00E94B006882396
:100FD00041F0209741F025E02A95F1F70000219794
:100FE000F4CFCD2B11F486E01FC082E390E00E9485
:100FF000B906892B11F487E017C00E94CC06892B13
:1010000019F0C2E3D0E009C088E00EC0209759F083
:1010100085E08A95F1F7000021970E94B0068823A9
:10102000A9F3CD2BB9F489E0809337018091370182
:101030008061809337010E949D060E94A306E19A79
:10104000E99A8FEF9FEFDF91CF911F910F91FF9062
:10105000EF9008958FEF9FEF90930301809302012B
:101060000E945E070E949D060E94A306E19AE99AEB
:10107000DF91CF911F910F91FF90EF900C94490752
:101080001F920F920FB60F9211242F933F934F93FD
:101090005F938F939F9329B1217080917303409147
:1010A0000001509101014115504819F48093360117
:1010B00012C090913601891771F09F5F891759F01E
:1010C00090E2909337018093360180E090E890930E
:1010D000010180930001809100019091010196959A
:1010E00087959093010180930001222349F080911C
:1010F000000190910101906890930101809300019B
:10110000809100019091010199278035910509F4A2
:1011100055C090F48031910509F450C020F4892B1A
:1011200009F4A0C067C08032910509F49BC08034E7
:10113000910509F497C05EC0803A910581F040F4B2
:101140008038910509F48EC080399105B9F152C0FB
:10115000803C910531F0803D910581F14BC084E6E2
:1011600013C08091000190910101892F99279093DC
:1011700001018093000183E02FC0882379F025E0EE
:101180002A95F1F700008150499BF7CF07C08823CB
:1011900049F095E09A95F1F7000081504999F7CF11
:1011A000811160C08091000190910101892F9927E0
:1011B000909301018093000182E00EC080910001B4
:1011C0009091010136E0969587953A95E1F79093D5
:1011D00001018093000181E080933801809100013A
:1011E0009091010199278F3F9105A1F48FEF809392
:1011F000370110C080E88093370180E090E8909339
:1012000001018093000180E09FEF909303018093A0
:10121000020128C080910201909103018827811565
:101220009F4F19F080E480933701809102019091E3
:101230000301982F88279093030180930201209146
:101240000001309101018091020190910301822BF4
:10125000909303018093020180E090E89093010154
:10126000809300019F918F915F914F913F912F91BA
:101270000F900FBE0F901F901895CF93C82F8DEE33
:101280000E946B078C2FCF910C946B07E82FE6958B
:10129000E695E695EF70F0E0EE5BFE4F4081282F7B
:1012A000277081E090E002C0880F991F2A95E2F72D
:1012B000242F30E028233923232B11F4842B80831F
:1012C0000895E82FE695E695E695EF70F0E0EE5B81
:1012D000FE4F2081382F377081E090E002C0880FE8
:1012E000991F3A95E2F7422F50E048235923452BA6
:1012F00019F08095822380830895482F50E0FA01E9
:101300003397E138F10508F048C0E65CFF4F0C94D4
:10131000292587E108958FE108958CE5089580E6F9
:10132000089582E6089587E2089583E508958FE29F
:10133000089589E3089587E308958FE3089587E486
:1013400008958FE4089586E508958EE508958FE663
:10135000089580E0089585E608958EE608958FE764
:10136000089580E3089588E3089580E4089588E46B
:10137000089580E5089587E508958FE5089588E14B
:10138000089588E0089580E2089580E1089589E154
:1013900008958DE6089588E208958F7708958FE087
:1013A0000895CF93482F50E0FA017C97E834F10577
:1013B000A0F5E554FF4F0C94292585E53EC08AE54C
:1013C0003CC08BE53AC08CE538C08DE536C08EE573
:1013D00034C08FE532C080E630C081E62EC082E6A0
:1013E0002CC083E62AC08FE628C081E726C082E7AA
:1013F00024C084E722C085E720C087E71EC088E7B5
:101400001CC08AE71AC08CE718C08FE716C080E7B7
:1014100014C089E712C08BE710C0C82F1F928F93AA
:1014200081E894E09F938F930E943F060F900F9066
:101430000F900F908C2F01C084E5CF9108950F93EA
:101440001F93CF93DF930E94DA228C010E94FA0649
:10145000EC01019631F4C8010E94F222843F9140D0
:10146000A8F3CE01DF91CF911F910F9108950E94B3
:10147000E0060C94EF068091720381608093720302
:10148000E2E4F1E0119281E0E235F807D9F708953E
:10149000E82FF0E0EE5BFE4F80810895E2E4F1E09A
:1014A000119281E0E235F807D9F70895982F8091DD
:1014B0003F01823049F492FB882780F990FD8260D9
:1014C00091FD84600C943D090895CF93DF93809142
:1014D0003701882311F1809137011F928F9382E0A9
:1014E00095E09F938F930E943F068091370180750E
:1014F0000F900F900F900F9071F480913E01893002
:1015000051F48CEF94E09F938F930E943F061092CA
:101510003E010F900F9010923701E0913E018E2F07
:1015200090E08A30910508F01FC3FC01ED5FFE4F8B
:101530000C9429250E94DA229F938F9387EF94E0E1
:101540009F938F930E943F0610923F01109241019A
:10155000109240010E944E0A0E94391881E035C065
:101560000E94F5062E98269A2F98279A0E94DA2232
:1015700090933D0180933C0182E00BC080913C013F
:1015800090913D010E94F222853F914008F4ECC207
:1015900083E080933E01E8C22E9826982F982798E2
:1015A0000E945E070E94EF060E94DA229F938F93AB
:1015B00082EF94E09F938F930E943F060E94DA226D
:1015C00090933D0180933C0184E080933E010F9015
:1015D0000F900F900F90C8C20E94FA06019609F46E
:1015E000C3C20E94DA229F938F938DEE94E09F9363
:1015F0008F930E943F060E94DA2290933D018093D0
:101600003C0185E0E2CF80913C0190913D010E9438
:10161000F222853F914018F087E080933E010E94BE
:10162000FA06019609F4A0C20E94DA229F938F93D2
:1016300088EE94E09F938F930E943F060E94DA22E7
:1016400090933D0180933C0186E0BFCF80913C01A7
:1016500090913D010E94F222853F914018F087E071
:1016600080933E010E94FA06019609F47DC20E9411
:10167000DA229F938F9383EE94E09F938F930E943F
:101680003F0687E0A2CF0E94DA229F938F938EEDD0
:1016900094E09F938F930E943F0682EF0E946B0716
:1016A0000F900F900F900F908F3F2FEF920789F0C0
:1016B0008A3F910589F40E941F0A8F3F3FEF9307ED
:1016C00071F0D82FCC270E941F0A9E01282BC90138
:1016D00008C08FEF9FEF05C08EEF9FEF02C080E044
:1016E00090E09093410180934001809137018823DD
:1016F00081F0809137011F928F9383ED94E09F9347
:101700008F930E943F06109237010F900F900F9019
:101710000F9080914001909141019C012227211559
:101720004BEA340711F482E00CC021153F4B11F451
:1017300083E007C00097B9F38F3F2FEF920721F4A2
:1017400081E080933F010DC08F3F910561F78DEBE4
:1017500094E09F938F930E943F0610923F010F9059
:101760000F9080913F011F928F93809141018F9341
:10177000809140018F9380EB94E09F938F930E9420
:101780003F0688E080933E010F900F900F900F90DE
:101790000F900F90E9C10E94DA229F938F938BEAFA
:1017A00094E09F938F930E943F060F900F900F90AD
:1017B0000F9080913F01823031F0833041F488EF07
:1017C0000E946B0704C00E94B1150E94560A89E06E
:1017D00080933E010E94DA229F938F9386EA94E0E1
:1017E0009F938F930E943F060F900F900F900F9042
:1017F000C0913F01C23009F47EC0C33009F439C141
:10180000C13009F0B1C10E94FA068F3F3FEF930744
:1018100009F4AAC19C012F7733272236310548F0FD
:101820008BE994E09F938F930E943F0610923B01B7
:1018300097C120913B01223009F444C028F42223AF
:1018400051F0213019F154C0233009F447C024303D
:1018500009F449C04DC0803E910569F01CF4009721
:1018600039F00EC0813E910549F08F3F910541F45A
:1018700080E994E071C1C0933B0176C182E02BC046
:101880008038910508F42BC18F7761C186339105AB
:1018900079F124F48A32910539F42AC08A3A910503
:1018A00039F1863B910521F18038910528F40E9499
:1018B000D1090E9446091CC08F770E94D1090E945D
:1018C000610916C08D31910529F08D39910581F49A
:1018D00084E001C083E080933B0146C185349105DB
:1018E00039F485E5FCC08534910511F485E52FC1F7
:1018F00010923B0139C10E94FA068F3F4FEF9407C7
:1019000009F432C1E0913A014E2F50E049305105BF
:1019100008F0ACC0FA01E35FFE4F0C942925803E2D
:10192000910569F18CF48338910569F12CF40097E5
:1019300071F586E794E0C1C08438910531F18A3AA7
:10194000910509F40FC123C0803F9105D1F02CF41B
:10195000813E9105E1F484E080C08C3F910509F45B
:1019600001C18F3F910599F40E944E0A8BE694E0E5
:101970009F938F930E943F0610923A01F1C082E03C
:101980006CC081E06AC082E05DC08FE65BC08038D9
:10199000910508F4A4C00E944E0A8FE594E0DCC0D3
:1019A0008935910509F462C0803F910521F08231AB
:1019B000910519F45BC083E050C010923A01803861
:1019C000910518F40E947D098AC00E944E0A85E59F
:1019D00094E0C2C08338910529F08438910521F440
:1019E0008FE642C082E040C010923A0180389105F3
:1019F00008F4ADC00E944E0A8BE494E0ADC0109292
:101A00003A018231910509F4AFC08935910509F495
:101A1000ABC08038910518F40E947D0998C00E94DF
:101A20004E0A8EE394E098C08431910529F0803FFE
:101A30009105E1F486E011C085E00FC0873791057C
:101A4000A9F480E00E94460911C0449779F487E028
:101A500004C0803F910551F488E080933A0184C02E
:101A60008737910519F480E00E94610910923A01CC
:101A70007BC00E94FA068F3F2FEF920709F474C0D3
:101A800020913901222319F0213079F16DC0843879
:101A9000910501F13CF4009771F083389105E1F470
:101AA00082E01DC0803F910589F08F3F9105A1F430
:101AB00088E294E051C083E394E09F938F930E9467
:101AC0003F060E944E0A0E94391831C081E080937F
:101AD00039014AC08FE703C08038910518F40E948D
:101AE000460942C08BE194E037C08338910511F17B
:101AF0007CF4009739F58DE094E09F938F930E94DA
:101B00003F060E944E0A0E943918109239010FC0F8
:101B10008438910589F08F3F9105A1F48FEF93E010
:101B20009F938F930E943F061092390119C00F9026
:101B30000F901AC082E001C08FE70E9461091092E5
:101B4000390112C0109239018038910518F40E94B1
:101B500061090AC085EF93E09F938F930E943F062F
:101B60000F900F9010923E0181E0DF91CF91089588
:101B70008091760208950895CF93DF9300D01F924D
:101B8000CDB7DEB720917C03243021F523E02983F3
:101B90009B838A8382E08093E9008FEF9091E80035
:101BA000815095FD06C095ED9A95F1F700008111E1
:101BB000F5CF8091E80085FF0DC040E050E063E084
:101BC00070E0CE0101960E941E128091E8008E778F
:101BD0008093E8000F900F900F90DF91CF910895C0
:101BE000CF93DF9300D01F92CDB7DEB720917C0357
:101BF000243029F522E02983805891099B838A8328
:101C00002093E9008FEF9091E800815095FD06C088
:101C100095ED9A95F1F700008111F5CF8091E800DC
:101C200085FF0DC040E050E063E070E0CE0101961A
:101C30000E941E128091E8008E778093E8000F903A
:101C40000F900F90DF91CF910895CF93DF93EC0128
:101C500090917C03943009F048C08091140188234E
:101C6000D9F0809115018823B9F09093E90081E8BB
:101C7000815049F09091E80095FD05C09AE29A954F
:101C8000F1F700C0F5CF8091E80085FF2EC040E05D
:101C900050E060E270E019C081E08093E90081E8E3
:101CA000815059F09091E80095FD07C0EFE3F1E015
:101CB0003197F1F700C00000F3CF8091E80085FF75
:101CC00014C040E050E068E070E0CE010E941E12B7
:101CD0008091E8008E778093E80080E2FE01A6E51F
:101CE000B2E001900D928A95E1F7DF91CF910895CE
:101CF000CF93C0915401C1110BC00E94E622643CF5
:101D000079408105910520F081E080935401C1E084
:101D10008C2FCF910895FF920F931F93CF93DF9352
:101D2000D82F0FB607FE83C080917C03843081F0EA
:101D30008091070190E001962091090130E0822313
:101D400093232091080130E08217930709F0C9C05E
:101D50000E94780E811110C08091070190E00196D9
:101D60002091090130E0822393232091080130E083
:101D70008217930709F0B5C00E94DA228C01C09146
:101D8000E900CF709091EC00892F817090FD80E880
:101D9000C82B83E08093E90085E0F82E8091EB006A
:101DA00085FD42C08091EB0080FF3EC08091EE0037
:101DB00087FF3AC08091080190910701981709F4B4
:101DC00057C09091E80095FF8AC0E0910501F0911D
:101DD0000601E80FF11D20818F5F90910901892391
:101DE000809308012093F1008091E80085FDE2CF07
:101DF0008091E80080FFDECF8091E8008E778093AD
:101E0000E800F0920401D6CF8091070190E001969E
:101E10002091090130E0822393232091080130E0D2
:101E20008217930709F448C0CF70C093E90040912E
:101E30000701842F90E001962091090130E0822370
:101E400093232091080130E08217930709F44CC0D6
:101E5000E0910501F0910601E40FF11DD08380911E
:101E600007018F5F909109018923809307013CC08E
:101E70008091E80085FF33C0D093F10081E090911C
:101E8000F200992391F09091E80090FF0EC090919C
:101E9000E80095FF03C01092F100F9CF9091E8009F
:101EA0009E779093E800F0920401882309F4ACCF68
:101EB000CF70C093E90018C080910401882309F411
:101EC000B3CF0E94DA229C018017910711F4890197
:101ED00065CF90910401915090930401F8CF80E078
:101EE000CECF40910701B4CF80E0DF91CF911F9119
:101EF0000F91FF9008950895089542E061EC81E00C
:101F00000E94971142E061EC82E00E94971142E248
:101F100061EC83E00E94971142E261EC84E00C9452
:101F2000971180917E03833009F455C030F48130DD
:101F300071F0823009F48EC008958A3009F47AC0B5
:101F40008B3009F460C0893009F09CC020C08091BA
:101F50007D03813A09F096C08091E800877F8093E5
:101F6000E8008091810390918203892B21F460E243
:101F700086E592E003C060E080E090E070E00E94BF
:101F80006B128091E8008B778093E8000895809130
:101F90007D03813209F076C08091810390918203A4
:101FA000009719F0039709F06DC08091E800877FD2
:101FB0008093E8008091E80082FD05C080917C0359
:101FC0008111F8CF5FC08091F100809376028091FB
:101FD000E8008B7753C080917D03813A09F052C0AD
:101FE0008091810390918203892B09F04BC08091ED
:101FF000E800877F8093E8008091E80080FFFCCFB5
:102000008091140136C080917D038132D9F5809191
:10201000810390918203892BA9F58091E800877F45
:102020008093E8000E94CC1180917F03809314017B
:102030000C94391880917D03813221F58091E8005C
:10204000877F8093E8000E94CC1180918003809369
:102050007702089580917D03813AA1F48091E80090
:10206000877F8093E8008091E80080FFFCCF80911B
:1020700077028093F1008091E8008E778093E800EA
:102080000C94CC11089580917602809355011092A2
:1020900076020E944E0A0C9439180C9443100E9448
:1020A000872280917A03882329F00E94942281114B
:1020B0000C94811108950E94A8228091550180936B
:1020C000760208950C945B1008950C946410CF93DD
:1020D00084B7877F84BF0FB6F894A895809160007D
:1020E000886180936000109260000FBE90E080E8ED
:1020F0000FB6F89480936100909361000FBE8BE857
:102100009EE00E945A228AE091E00E94AC1581E391
:1021100095E00E94A6050E94370A0E9460160E9460
:1021200084140E94D7148091E20084608093E200BE
:1021300078940E94621680917C03843029F00E947A
:1021400091150E946410F7CF8FE195E00E94A605DB
:102150000E9465108DE095E00E94A605C3E0809185
:102160007C03853019F40E944F10F9CF0E94661647
:102170002091E4003091E50080915201909153014B
:102180002817390709F464C08091E4009091E500B4
:1021900090935301809352010E94780E882309F492
:1021A00057C080917C03843009F052C08091E900CF
:1021B0008F702091EC00922F917020FD90E8892B78
:1021C000C093E9009091EB0090FF3FC09091EE002A
:1021D00097FF3BC09091080120910701291709F151
:1021E0002091E80025FF1DC0E0910501F091060156
:1021F000E90FF11D30819F5F209109019223909397
:1022000008013093F1009091E80095FDE3CF9091A3
:10221000E80090FFDFCF9091E8009E779093E80070
:10222000D9CF9091F200992381F09091E80090FF2E
:102230000CC09091E80095FF03C01092F100F9CF17
:102240009091E8009E779093E8008F708093E9006A
:102250000E94911584CF292F332723303105C9F0EF
:1022600060F42130310581F02230310509F041C0A0
:1022700084E790E021E935E040C021323105E1F00A
:102280002232310531F135C082E190E025E036E0BF
:1022900034C099278130910549F028F0029749F51B
:1022A000E7E4F5E005C0EDE8F5E002C0EDE7F5E0B4
:1022B000849190E09F0121C064307105D0F4660FD5
:1022C000771FFB01EC5DFE4F2081318189E090E0BA
:1022D00014C06430710568F4FB01EE0FFF1FE45E6B
:1022E000FE4F20813181FB01E85EFE4F808190E04E
:1022F00004C080E090E020E030E0FA0131832083E8
:10230000089584E089BD86E089BD09B400FEFDCF53
:102310008091D8008F7D8093D8008091E00082600A
:102320008093E0008091E00081FDFCCF0895982F1C
:10233000953068F59093E900981739F07091EC00AA
:102340002091ED005091F00003C0242F762F50E033
:1023500021FD02C09F5FECCF3091EB003E7F3093B8
:10236000EB003091ED003D7F3093ED003091EB00BC
:1023700031603093EB007093EC002093ED005093AC
:10238000F0002091EE0027FDE5CF80E008958F70EA
:102390008093E90081E0089580917D0387FF11C05B
:1023A0008091E80082FD05C080917C038111F8CF07
:1023B00011C08091E8008B770BC080917C0388234B
:1023C00049F08091E80080FFF8CF8091E8008E7797
:1023D0008093E80008952091E4003091E50095E6AF
:1023E0004091EC00842F817040FF23C08091E80071
:1023F00080FD1DC080917C03882399F0853099F081
:102400008091EB0085FD11C04091E4005091E50002
:102410002417350729F3915011F09A01E1CF84E098
:10242000089582E0089583E0089581E0089580E0B2
:1024300008954091E80042FFDDCF0895CF92DF92EA
:10244000EF92FF920F931F93CF93DF93EC018B01D9
:102450007A010E94EB11811135C0E114F10439F0C9
:10246000F70180819181081B190BC80FD91FC12C5E
:10247000D12C0115110529F18091E80085FD18C0C6
:102480008091E8008E778093E8000E949115E11416
:10249000F10449F0F70180819181C80ED91ED182E3
:1024A000C08285E00FC00E94EB11882311F30AC09F
:1024B00089918093F10001501109FFEFCF1ADF0AD3
:1024C000D8CF80E0DF91CF911F910F91FF90EF90D7
:1024D000DF90CF90089520918303309184032617D5
:1024E000370748F06115710539F42091E8002E771F
:1024F0002093E80001C0B901FC0120E061157105DD
:1025000061F180917C038823D9F18530D9F18091E4
:10251000E80083FD39C08091E80082FD2BC08091E6
:10252000E80080FFEBCF8091F20090E0611571052B
:1025300051F08830910538F421912093F1006150D9
:1025400071090196F3CF21E0089709F020E080910E
:10255000E8008E778093E800D1CF2111D2CF0AC056
:1025600080917C03882361F0853061F08091E800E0
:1025700083FD0AC08091E80082FFF2CF80E00895D9
:1025800082E0089583E0089581E008952091830317
:10259000309184032617370748F06115710539F427
:1025A0002091E8002E772093E80001C0B901FC01DA
:1025B00020E06115710579F180917C03882309F48D
:1025C0003DC0853009F43CC08091E80083FD3AC0ED
:1025D0008091E80082FD2CC08091E80080FFE9CF67
:1025E0008091F20090E06115710559F088309105F5
:1025F00040F424912093F1003196615071090196C5
:10260000F2CF21E0089709F020E08091E8008E7772
:102610008093E800CECF2111CFCF0AC080917C03F8
:10262000882361F0853061F08091E80083FD0AC065
:102630008091E80082FFF2CF80E0089582E0089563
:1026400083E0089581E008951F93CF93DF93CDB782
:10265000DEB7AA970FB6F894DEBF0FBECDBFEDE789
:10266000F3E08091F100819323E0E538F207C9F7A8
:102670000E94910F8091E80083FF2EC180917D031D
:1026800090917E03492F50E04A30510508F024C153
:10269000FA01EA5EFE4F0C942925803821F0823839
:1026A00009F01AC108C08091790390917A039923A7
:1026B00089F082600FC0809181038F70853008F0AF
:1026C0000BC18093E9008091EB0085FB882780F99E
:1026D0001092E9009091E800977F9093E800809332
:1026E000F1001092F100D1C0282F2D7F09F0F4C025
:1026F000882319F0823061F0EFC080917F03813030
:1027000009F0EAC0933009F080E080937A032EC08C
:1027100080917F0381112AC0809181038F702FEFF8
:10272000280F243008F0D8C08093E9002091EB00F6
:1027300020FF1CC0933021F48091EB00806214C014
:102740009091EB0090619093EB0021E030E0A901C3
:1027500002C0440F551F8A95E2F74093EA00109299
:10276000EA008091EB0088608093EB001092E90012
:102770008091E800877F8093E8000E94CC11ACC074
:102780008111AAC010917F031F778091E3008078A8
:10279000812B8093E3008091E800877F8093E8009D
:1027A0000E94CC118091E80080FFFCCF8091E30073
:1027B00080688093E300111102C082E001C083E0D1
:1027C00080937C0389C08058823008F085C0809156
:1027D0007F03909180038C3D53E0950779F583E06A
:1027E0008A838AE289834FB7F894DE01139620E04A
:1027F0003EE051E2E32FF0E050935700E49120FFD8
:1028000003C0E295EF703F5FEF708E2F90E0EA30EB
:1028100010F0C79601C0C0968D939D932F5F243111
:1028200049F74FBF8091E800877F8093E8006AE214
:1028300070E0CE0101960E946B1216C06091810378
:1028400070918203AE014F5F5F4F0E942B11BC015C
:10285000892B09F441C09091E800977F9093E8009C
:1028600089819A810E94C6128091E8008B778093BB
:10287000E80032C0803881F58091E800877F80933E
:10288000E800809178038093F1008091E8008E77D2
:1028900072CF811121C080917F039091800399278D
:1028A0000297D4F48091E800877F8093E8008091BC
:1028B0007F03809378030E94CC118091780381116B
:1028C00006C08091E30087FD02C081E001C084E082
:1028D00080937C030E947D0F8091E80083FF0AC0F3
:1028E0008091E800877F8093E8008091EB00806210
:1028F0008093EB00AA960FB6F894DEBF0FBECDBF53
:10290000DF91CF911F9108950E94E1140E94E41479
:10291000E0EEF0E0808181608083E8EDF0E080818E
:102920008F77808319BCE3E6F0E08081816080834B
:1029300010927B0308950E94E1140E94E414809198
:10294000D8008F778093D8008091D80080688093DA
:10295000D8008091D8008F7D8093D80084E089BD15
:1029600086E089BD09B400FEFDCF10927C03109271
:10297000780310927A031092790342E060E080E0DD
:102980000E9497118091E1008E7F8093E1008091F9
:10299000E20081608093E2008091E2008860809391
:1029A000E2008091E0008E7F8093E0000895E3E6EE
:1029B000F0E080818E7F808381E080937B030C94A4
:1029C0009B141092E20008951092E10008951F9266
:1029D0000F920FB60F9211242F933F934F935F9353
:1029E0006F937F938F939F93AF93BF93EF93FF93D7
:1029F0008091E10082FF0BC08091E20082FF07C05E
:102A00008091E1008B7F8093E1000E947C0F809198
:102A1000E10080FF19C08091E20080FF15C0809125
:102A2000E2008E7F8093E2008091E20080618093DB
:102A3000E2008091D80080628093D80019BC85E0C4
:102A400080937C030E944D108091E10084FF30C090
:102A50008091E20084FF2CC084E089BD86E089BDBE
:102A600009B400FEFDCF8091D8008F7D8093D800FF
:102A70008091E1008F7E8093E1008091E2008F7E63
:102A80008093E2008091E20081608093E200809177
:102A90007803882311F084E007C08091E30087FD6C
:102AA00002C081E001C083E080937C030E94621039
:102AB0008091E10083FF24C08091E20083FF20C069
:102AC0008091E100877F8093E10082E080937C0326
:102AD000109278038091E1008E7F8093E1008091D5
:102AE000E2008E7F8093E2008091E200806180931B
:102AF000E20042E060E080E00E9497110E947B0FBC
:102B0000FF91EF91BF91AF919F918F917F916F91C5
:102B10005F914F913F912F910F900FBE0F901F909B
:102B20001895CF9380917C038823A1F0C091E90090
:102B3000CF709091EC00892F817090FD80E8C82BB8
:102B40001092E9008091E80083FD0E942413CF7069
:102B5000C093E900CF91089590937D0280937C0209
:102B60000895E0917C02F0917D02309721F0019070
:102B7000F081E02D099480E00895EF92FF920F9389
:102B80001F93CF93DF93E0917C02F0917D02309709
:102B9000B1F18C010280F381E02D099580917203DF
:102BA00082FF2DC080FF04C08EE097E00E94A60542
:102BB000E80110E288E0E82E87E0F82E80917203A9
:102BC00080FF0BC088811F928F93FF92EF920E942B
:102BD0003F060F900F900F900F90115021961111FA
:102BE000EDCF8091720380FF0AC086E097E0DF910D
:102BF000CF911F910F91FF90EF900C94A605DF915C
:102C0000CF911F910F91FF90EF900895CF93DF9395
:102C100020917A0230917B022817390709F19093AD
:102C20007B0280937A02E0917C02F0917D023097E2
:102C3000B9F0EC010680F781E02D099580917203CF
:102C400082FF0EC080FF0CC0DF93CF9388EF96E029
:102C50009F938F930E943F060F900F900F900F90BD
:102C6000DF91CF910895CF93DF9320917802309137
:102C700079022817390709F1909379028093780235
:102C8000E0917C02F0917D023097B9F0EC01008474
:102C9000F185E02D09958091720382FF0EC080FFBF
:102CA0000CC0DF93CF9388EE96E09F938F930E94A2
:102CB0003F060F900F900F900F90DF91CF910895E6
:102CC0000C9409170E94D1220C943B0ABF92CF9218
:102CD000DF92EF92FF920F931F93CF93DF9300D079
:102CE00000D01F92CDB7DEB70E94650A0FE712E051
:102CF000F12C8F2D0E94480AB82EF801C080C826FA
:102D000039F4F3940F5F1F4FF0E1FF12F2CF30C0A0
:102D10008091720381FD0E940A17D12CEE24E39466
:102D20008C2D8E21F9F0D982FA8291E08B2D8E21A3
:102D300009F490E09B830E94DA228160782F9D83C2
:102D40008C8349815A816B818D810E944017498112
:102D50005A816B817C818D810E947222F801808171
:102D60008E258083D394EE0CF8E0DF12D9CFC9CF43
:102D70008FEF89838A831B820E94DA228160782FF9
:102D80009D838C8349815A816B818D810E9440177C
:102D90000E9471220E94B11590917E02891741F123
:102DA0000E94B11580937E029091720392FF0EC033
:102DB00090FF0CC01F928F9389E197E09F938F93B0
:102DC0000E943F060F900F900F900F9080917E020F
:102DD0000F900F900F900F900F90DF91CF911F9158
:102DE0000F91FF90EF90DF90CF90BF900C948322D3
:102DF0000F900F900F900F900F90DF91CF911F9138
:102E00000F91FF90EF90DF90CF90BF9008950C94BA
:102E1000560A0895EF92FF920F931F93CF93DF937B
:102E200082E397E00E94A605C0E0D0E08CE2E82EA5
:102E300081E0F82E04E217E08C2F0E94480A0E94DD
:102E40005F22FF92EF921F928F93DF93CF931F9396
:102E50000F930E943F0621968DB79EB708960FB636
:102E6000F8949EBF0FBE8DBFC031D10529F7DF9109
:102E7000CF911F910F91FF90EF90089508950895BD
:102E8000CF93DF93CDB7DEB72B970FB6F894DEBFA5
:102E90000FBECDBF942F4F83252F588769877A8720
:102EA0008B874A855B85452B31F02F3F31F481E0DC
:102EB0009F3F19F403C081E001C080E080FD07C09E
:102EC0004F81588569857A858B850E947222DE0143
:102ED000119686E0FD0111928A95E9F785E0FE01E1
:102EE000379601900D928A95E1F749815A816B815D
:102EF0007C818D819E810E94611E2B960FB6F89475
:102F0000DEBF0FBECDBFDF91CF910895CF93882351
:102F100009F465C0C82F8CEF8C0F813A20F080E552
:102F20008C0F8E3248F48C2F0E94C524811157C01B
:102F30008C2F0E9455210CC080E28C0F883058F4F1
:102F4000C77081E001C0880FCA95EAF70E94FA2194
:102F5000CF910C9434228BE58C0F833078F4C53AF2
:102F600029F0C63A31F083E890E005C081E890E0AE
:102F700002C082E890E0CF910C94061688E58C0F91
:102F8000853168F5C83A89F0C93A91F0CA3A99F0A2
:102F9000CB3AA1F0CC3AA9F0CD3AB1F0CE3AB9F0A3
:102FA000CF3AC1F080E090E017C082EE90E014C00C
:102FB00089EE90E011C08AEE90E00EC085EB90E0C3
:102FC0000BC086EB90E008C083EB90E005C084EB7B
:102FD00090E002C087EB90E0CF910C943316CF9134
:102FE0000895882349F19CEF980F913A20F090E5DD
:102FF000980F9E3218F40E94A5210DC090E2980F00
:10300000983058F4877091E001C0990F8A95EAF7DB
:10301000892F0E9400220C9434229BE5980F933054
:1030200020F480E090E00C940616885A853120F454
:1030300080E090E00C9433160895882321F00E94DC
:10304000FA210C9434220895882321F00E94002252
:103050000C94342208950E941A220E94E9210E94B1
:10306000342280E090E00E94061680E090E00C940C
:1030700033160E940A220C942B18CF92DF92EF9203
:10308000FF920F931F93CF93DF9300D000D01F9236
:10309000CDB7DEB76C010E9485228111EAC285E0BE
:1030A000F601DE01119601900D928A95E1F7F60185
:1030B00040815181238134812115310531F05F3FF9
:1030C00031F481E04F3F19F403C081E001C080E09A
:1030D00080FDCFC2F601F280E580E2948FE0E82225
:1030E00049835A83FB82722F3D832C836F2D8D8100
:1030F0000E94CA208C010E94C9200E94B91FE12FA2
:10310000E295EF708E2F90E0FC01E05EFE4F0C9494
:103110002925812F807F1F70882311F01295107F41
:10312000FF2049F0112309F43BC2812F0E940D2298
:103130000E94342235C2802F0E94F117112309F416
:1031400098C2812F0E9413220F900F900F900F9022
:103150000F90DF91CF911F910F91FF90EF90DF9033
:10316000CF900C943422812F807F1F70803211F019
:103170001295107F002319F0013009F12BC0FF20B8
:10318000A9F0EE2059F1F1E0812FEF1228C00F9045
:103190000F900F900F900F90DF91CF911F910F9193
:1031A000FF90EF90DF90CF900C941D22EE2021F045
:1031B00021E0E21609F45DC20E9420222DC0FF200A
:1031C000E9F085E08E1508F454C20E94F7218123AE
:1031D00029F022C0FF20F1F0E11015C0812F0F90DF
:1031E0000F900F900F900F90DF91CF911F910F9143
:1031F000FF90EF90DF90CF900C941D1894E09E15F7
:1032000008F437C209C0F601858180FFC9C18F70FB
:103210008583E4CFE110D7C1812F4AC1812F8695E4
:103220008695837019F08130B9F023C2FF2019F020
:10323000C801937002C080E090E00F900F900F9053
:103240000F900F90DF91CF911F910F91FF90EF9012
:10325000DF90CF900C940616FF2019F0C8019370F0
:1032600002C080E090E00F900F900F900F900F90B1
:10327000DF91CF911F910F91FF90EF90DF90CF9052
:103280000C943316812F837009F070C0F110F1C1D6
:10329000202F229526952770220F220F602F6F7006
:1032A000862F90E0A0E0B0E06C017D01022E04C00A
:1032B000CC0CDD1CEE1CFF1C0A94D2F704FF12C0DC
:1032C0008FE090E0A0E0B0E004C0880F991FAA1F33
:1032D000BB1F2A95D2F7BC01CD01609570958095F2
:1032E000909503C060E070E0CB01169516951370C1
:1032F0001230B1F040F56C297D298E299F291130BB
:1033000031F10F900F900F900F900F90DF91CF91B0
:103310001F910F91FF90EF90DF90CF900C94DE1FE4
:103320006C297D298E299F290F900F900F900F9067
:103330000F90DF91CF911F910F91FF90EF90DF9051
:10334000CF900C94F81F0E94DE1FC701B6010F90AA
:103350000F900F900F900F90DF91CF911F910F91D1
:10336000FF90EF90DF90CF900C94C41FFF2019F0D6
:10337000812F817001C08695882309F47AC1202F9E
:10338000229526952770220F220F602F6F70862FAF
:1033900090E0A0E0B0E06C017D01022E04C0CC0CF6
:1033A000DD1CEE1CFF1C0A94D2F704FF12C08FE054
:1033B00090E0A0E0B0E004C0880F991FAA1FBB1FD7
:1033C0002A95D2F7BC01CD016095709580959095B6
:1033D00003C060E070E0CB011695169513701230B3
:1033E000B1F040F56C297D298E299F29113031F1EA
:1033F0000F900F900F900F900F90DF91CF911F9132
:103400000F91FF90EF90DF90CF900C94A5206C2946
:103410007D298E299F290F900F900F900F900F906C
:10342000DF91CF911F910F91FF90EF90DF90CF90A0
:103430000C94B7200E94A520C701B6010F900F90F1
:103440000F900F900F90DF91CF911F910F91FF90F0
:10345000EF90DF90CF900C949320003FC1F128F4BF
:1034600080E4800F803250F096C0023F09F45EC0C5
:1034700008F449C0033F09F46CC08DC0F02FF0710F
:10348000EF2E812F8F71FF2051F00E942C20802F72
:10349000EE2019F08295807FA2CE8F70A0CE0E9480
:1034A0004D20802FEE2019F08295807F01C08F7013
:1034B0000F900F900F900F900F90DF91CF911F9171
:1034C0000F91FF90EF90DF90CF900C942418FF2085
:1034D000A9F024E02E1508F4CCC0812F8F710F9035
:1034E0000F900F900F900F90DF91CF911F910F9140
:1034F000FF90EF90DF90CF900C94722085E08E15B6
:1035000008F4B7C0EACFFF2099F0812F8F710F9098
:103510000F900F900F900F90DF91CF911F910F910F
:10352000FF90EF90DF90CF900C942C20FF2069F358
:10353000812F8F710F900F900F900F900F90DF9150
:10354000CF911F910F91FF90EF90DF90CF900C944F
:103550004D20FF2089F0812F8F710F900F900F90D9
:103560000F900F90DF91CF911F910F91FF90EF90EF
:10357000DF90CF900C9417200F900F900F900F902A
:103580000F90DF91CF911F910F91FF90EF90DF90FF
:10359000CF900C941220FF2099F0EE2009F4B5CFC3
:1035A000802F0F900F900F900F900F90DF91CF9181
:1035B0001F910F91FF90EF90DF90CF900C948617A2
:1035C000EE2009F4B5CF802F0F900F900F900F9041
:1035D0000F90DF91CF911F910F91FF90EF90DF90AF
:1035E000CF900C94F117412F4F70602FC6010E94AD
:1035F00060230F900F900F900F900F90DF91CF915D
:103600001F910F91FF90EF90DF90CF900C94141FBB
:1036100001112FC0FF2069F10E9439189FEFE0E7E8
:10362000F2E09150E040F040E1F700C000000F9060
:103630000F900F900F900F90DF91CF911F910F91EE
:10364000FF90EF90DF90CF900C944123412F4F706B
:10365000602FC6010F900F900F900F900F90DF9189
:10366000CF911F910F91FF90EF90DF90CF900C942E
:1036700063230F900F900F900F900F90DF91CF91D9
:103680001F910F91FF90EF90DF90CF9008951F93BF
:10369000CF93DF9300D000D01F92CDB7DEB7942F29
:1036A0004983252F5A836B837C838D834C815D8175
:1036B000452B31F02F3F31F481E09F3F19F403C0D7
:1036C00081E001C080E0182F117080FD31C0498178
:1036D0005A816B817C818D810E94CA20292F22957D
:1036E0002F702C3030F42A30A0F42250223030F0E9
:1036F00022C02C30C9F02F30B9F01DC0853A28F413
:103700008430C0F4823028F415C090E2980F9830CD
:1037100088F0883E30F4803E68F48450813A58F452
:1037200009C0803F41F406C093FB112710F903C084
:1037300010E001C011E0812F0F900F900F900F90BB
:103740000F90DF91CF911F910895CF93DF9300D019
:1037500000D01F92CDB7DEB70F900F900F900F9053
:103760000F90DF91CF910895CF93DF9300D000D0D9
:1037700000D0CDB7DEB726960FB6F894DEBF0FBEE9
:10378000CDBFDF91CF910895CF93DF93C0918F028A
:1037900080919002C817A1F0D0E0CE0166E070E001
:1037A0000E941825FC01EF56FD4F40815181628136
:1037B0007381848195810E94B41B2196C770E8CFE4
:1037C000DF91CF9108954091C1025091C202609162
:1037D000C3027091C4028091C5029091C6020C94FC
:1037E000B41B1F93CF93DF938091C60282958F7095
:1037F00009F066C08091C302882309F461C020915A
:103800008F0210919002C091C102D091C202E0914A
:10381000C402F091C50281E0CF3F09F080E0482F5B
:10382000211709F44DC0309721F0DF3F21F080E0EF
:1038300003C081E001C0842F30E080FD3DC0C9019C
:1038400066E070E00E941825DC01AF56BD4F11966E
:103850008C9111978D1330C08C918C132DC01296C2
:103860008C911297811128C013968D919C91149779
:103870008E179F0708F401978E1B9F0B883C9105BC
:10388000D8F48091C6028F7080618093C602C9010E
:1038900066E070E00E941825FC01EA56FD4F908119
:1038A0009F709061908381EC92E00E943D18DF91BF
:1038B000CF911F910C94C41B2F5F3F4F2770B0CF47
:1038C000DF91CF911F910895AF92BF92CF92DF9277
:1038D000EF92FF920F931F93CF93DF93CDB7DEB795
:1038E00061970FB6F894DEBF0FBECDBF7C0185E0B7
:1038F000F701DE011D9601900D928A95E1F7D7013F
:103900004C9111962C9111971296DC901297139668
:103910000D911C9114975091C1026091C202809147
:10392000C4029091C502009731F06F3F31F431E04D
:103930005F3F19F403C031E001C030E0B32FB17034
:10394000BB2E30FD76C1A090C302AA2009F4D2C0DC
:103950003091C6020817190728F0F801E81BF90B87
:10396000CF0104C080959095800F911FCC24C39403
:10397000883C910588F0C12C307F09F0A6C0702FDB
:10398000198B088B522F6D2D89890E94A51B81EC04
:1039900092E00E943D18C3C0832F807F09F059C078
:1039A000261315C0451313C0CD2CD11010C03F7085
:1039B00030613093C6020E94E31B81EC92E00E94CA
:1039C0003D188091C602D70115968C9368C10115E8
:1039D000110531F02F3F31F481E04F3F19F403C05E
:1039E00081E001C080E080FD03C081E08D2502C040
:1039F00080E090E0B82FB170CB2E80FF1FC0E09127
:103A00008F0230919002E31709F425C1F0E0CF0155
:103A100066E070E00E941825DC01AF56BD4F11969C
:103A20008C911197281307C08C91481304C01296EB
:103A30008C91D81203C03196E770E5CFCD2CDD20F4
:103A400009F42DC18091C60281608093C602C12C09
:103A500026C1261308C0451306C0D11004C08091AA
:103A6000C602D701B9C04D872E87DF86702F198B0C
:103A7000088B522F6D2D89890E94471B8823A1F145
:103A8000DD2091F12091C602822F82958F7090E007
:103A9000029774F08091C1029091C20298878F833F
:103AA00019861B870A872C87CE0107960E943D182E
:103AB00086E0F701A1ECB2E001900D928A95E1F762
:103AC0000E94F11B0E94E31B12C0261791F14D8743
:103AD0002E87DF86702F198B088B522F6D2D8989C9
:103AE0000E94471B811139C0C7010E943D18CC2498
:103AF000C394D5C00817190708F447C0F801E81B9C
:103B0000F90BCF01883C910508F444C0C12C702FFB
:103B1000198B088B522F6D2D89890E94A51BE1EC12
:103B2000F2E086E0DF011D928A95E9F70E94E31B2F
:103B3000B6C04513CCCFD110CACF8091C602F701D1
:103B40008583C7010E943D1886E0E1ECF2E0DF01C9
:103B50001D928A95E9F7CA2CA2C0DD2029F2209196
:103B6000C602822F82958F7090E002970CF4A0CF4E
:103B70008091C1029091C2029A8389831B821D8326
:103B80000C832E83CE01019691CF80959095800F66
:103B9000911FB8CFCD2CDD2009F4A6CF261333C05A
:103BA000451331C02091C60220FD24C0822F82958A
:103BB0008F70482F50E041155105E1F0D70115965F
:103BC0002C9315974F30510549F08F5F982F9295A0
:103BD000907F822F8F70892B15968C93C7010E943E
:103BE0003D1886E0F701A1ECB2E001900D928A95B4
:103BF000E1F79CCF86E0F701A1ECB2E001900D92D5
:103C00008A95E1F74CC04D872E87DF86702F198B80
:103C1000088B522F6D2D89890E94471B811148CF37
:103C20008091C60281608093C602C7010E943D1840
:103C300036C0DD2009F458CF4D872E87DF86702FE0
:103C4000198B088B522F6D2D89890E94471B882361
:103C500009F44ACF2DCF702F198B088B522F6D2D61
:103C600089890E94CA20292F22952F70223028F49A
:103C70009F7039F0811105C00BC0243028F49F706B
:103C800049F4805E883020F0C7010E943D18BC2CAA
:103C9000CB2C05C0F7019581907F99F7F9CF8C2D3A
:103CA00061960FB6F894DEBF0FBECDBFDF91CF9106
:103CB0001F910F91FF90EF90DF90CF90BF90AF904A
:103CC0000895CF93DF93CDB7DEB72C970FB6F89456
:103CD000DEBF0FBECDBF4F83588769877A878B873A
:103CE0009C87CE0107960E94641C8823D1F09F8197
:103CF00088852A853B85232B31F08F3F31F481E085
:103D00009F3F19F403C081E001C080E080FD6FC0D7
:103D10004F81588569857A858B859C850E94B41B67
:103D200066C086E0FE013796DE01119601900D9285
:103D30008A95E1F7FF81E8856A857B8561157105C4
:103D400031F0EF3F31F481E0FF3F19F403C081E02F
:103D500001C080E080FD4BC08091900290E09C010A
:103D60002F5F3F4F2770332740918F0250E0241779
:103D7000350709F443C0F983EA837D836C8366E0E9
:103D800070E00E941825DC01AF56BD4F96E0FE01A1
:103D9000319601900D929A95E1F7209390020E943E
:103DA000C41B25C090E066E070E00E9418258F5685
:103DB0009D4F0E94641C882371F180918F0290E0D6
:103DC00066E070E00E941825FC01EF56FD4F40812F
:103DD000518162817381848195810E94B41B80919D
:103DE0008F0290E001968770992780938F028091CF
:103DF0008F02909190028913D5CF0DC00E9439187F
:103E00001092900210928F02E1ECF2E086E0DF0166
:103E10001D928A95E9F72C960FB6F894DEBF0FBE77
:103E2000CDBFDF91CF910895DF92EF92FF920F9374
:103E30001F93CF93DF93FC01892B09F488C0E12CF9
:103E4000F12CDD24D394EF0121968491853709F478
:103E500060C058F4843708F04EC0843008F068C061
:103E60008130D1F0823071F172C0883709F45BC0C3
:103E700050F4863709F453C0873709F068C08E2D97
:103E80000E94072252C09CE7980F903708F05FC04D
:103E90008F770E94F1174EC08F010E5F1F4FFE01FA
:103EA000849190E2980F983050F48770FD2D01C0F6
:103EB000FF0F8A95EAF78F2F0E940D2215C00E94EE
:103EC000861714C08F010E5F1F4FFE01849190E290
:103ED000980F983068F48770FD2D01C0FF0F8A9508
:103EE000EAF78F2F0E9413220E943422E80122C099
:103EF0000E94F117FBCFCF010296FE01C491CC23A3
:103F000061F0EFE9FFE03197F1F700C00000C15028
:103F1000F6CFCF010296FE01F490EC010BC00E9497
:103F2000F721E82E07C00E940A220E94342202C014
:103F30000E9486178F2D882341F0EFE9FFE031972B
:103F4000F1F700C000008150F6CFFE017CCFDF9179
:103F5000CF911F910F91FF90EF90DF9008956093A4
:103F60004703709348038093490390934A030C944A
:103F70008222089560934B0370934C0380934D030A
:103F800090934E030C9481220F931F9300914B0347
:103F900010914C0320914D0330914E03602B712BF7
:103FA000822B932B60934B0370934C0380934D03B0
:103FB00090934E031F910F910C9481220F931F93A6
:103FC00000914B0310914C0320914D0330914E030F
:103FD000602371238223932360934B0370934C03DC
:103FE00080934D0390934E031F910F910C94812267
:103FF0000F931F9300914B0310914C0320914D039D
:1040000030914E03602771278227932760934B03DB
:1040100070934C0380934D0390934E031F910F9127
:104020000C94812260E070E0CB010C94AF1F0F93E1
:104030001F9341E050E060E070E08A019B0104C002
:10404000000F111F221F331F8A95D2F7C901B80133
:104050001F910F910C94AF1F0F931F9341E050E0FD
:1040600060E070E004C0440F551F661F771F8A95FB
:10407000D2F78091470390914803A0914903B091F2
:104080004A038A019B01082B192B2A2B3B2BC901C0
:10409000B8011F910F910C94AF1F0F931F9341E034
:1040A00050E060E070E004C0440F551F661F771FAA
:1040B0008A95D2F740955095609570958091470309
:1040C00090914803A0914903B0914A038A019B0152
:1040D000082319232A233B23C901B8011F910F91FB
:1040E0000C94AF1F0F931F9341E050E060E070E02D
:1040F00004C0440F551F661F771F8A95D2F7809121
:10410000470390914803A0914903B0914A038A0163
:104110009B01082719272A273B27C901B8011F91AE
:104120000F910C94AF1F0F931F93009147031091B1
:1041300048032091490330914A03602B712B822B55
:10414000932B1F910F910C94AF1F0F931F9300910E
:104150004703109148032091490330914A0360239B
:104160007123822393231F910F910C94AF1F0F9300
:104170001F93009147031091480320914903309108
:104180004A0360277127822793271F910F910C9470
:10419000AF1F08958F929F92AF92BF92DF92EF92DE
:1041A000FF920F931F93CF93DF9300D000D01F9205
:1041B000CDB7DEB76B837C838D838A018C819D8133
:1041C000892B31F01F3F31F481E04F3F19F403C0D8
:1041D00081E001C080E080FF03C080E090E054C037
:1041E0008B81882309F43DC0809047039090480359
:1041F000A0904903B0904A0380914B0390914C03E7
:10420000A0914D03B0914E03882A992AAA2ABB2A6D
:104210002FE1E22EF12CD501C4010E2C04C0B6957D
:10422000A795979587950A94D2F780FD06C081E0FF
:10423000E81AF10880F7D12C07C0DE2CB8018E2DCA
:104240000E944806019799F3E12FF0E093E0EE0F0A
:10425000FF1F9A95E1F7E953FD4FE00FF11DD08262
:104260000CC0E12FF0E083E0EE0FFF1F8A95E1F72D
:10427000E953FD4FE00FF11DD08009831A83698156
:104280007A818D2D0E9448060F900F900F900F900D
:104290000F90DF91CF911F910F91FF90EF90DF90E2
:1042A000BF90AF909F908F900895909114019923A3
:1042B00079F190911501992359F1982F969596953A
:1042C00096959F31A1F0E0911601F0911701E90F49
:1042D000F11D877021E030E0A90102C0440F551F95
:1042E0008A95E2F7CA019181892B81830895909183
:1042F000720390FF29C01F928F938EE597E09F93E2
:104300008F930E943F060F900F900F900F9008958B
:104310002091160130911701F90132969FEF40E08C
:104320005191851789F09F3F19F4511101C0942FC5
:104330004F5F4E31A9F79F3F39F0F901E90FF11DA9
:1043400097FDFA9582830895089590911401992319
:1043500081F190911501992361F1982F9695969589
:1043600096959F31A9F0E0911601F0911701E90FA0
:10437000F11D877021E030E0A90102C0440F551FF4
:104380008A95E2F7CA0180959181892381830895F6
:104390009091720390FF1CC01F928F9380E497E06E
:1043A0009F938F930E943F060F900F900F900F9056
:1043B0000895E0911601F09117019F01225E3F4F91
:1043C0009281891301C012823196E217F307C1F777
:1043D000089581E090E0E0911601F0911701E80F57
:1043E000F91F1082019680329105A9F708958091F6
:1043F0007103089590917103892B8093710308953F
:10440000809590917103892380937103089580931F
:104410007103089510927103089590917003892B90
:104420008093700308958095909170038923809301
:104430007003089510927003089580934F030895B8
:1044400010924F0308958091160190911701FC017D
:1044500031969C01205E3F4F80E0919191118F5FDA
:10446000E217F307D1F70895E0911601F0911701D3
:10447000809171038083E0911601F0911701908182
:1044800080917003892B808380914F03882361F092
:10449000E0911601F09117019081892B80830E9491
:1044A0002322811110924F038091160190911701E0
:1044B0000C94BD1590933501809334010895829535
:1044C000982F9373292F220F220F982F9C7C96955B
:1044D0009695922B892F8575880F9A7A9695892BB8
:1044E00008950895CF93DF9300D000D01F92CDB7E9
:1044F000DEB70F900F900F900F900F90DF91CF913C
:104500000895089508950C94071780E0089583B7DF
:10451000817F8C6083BF83B7816083BF78948895E7
:1045200083B78E7F83BF0895CF930E943E170E946A
:10453000650A0E943F17C0E08C2F0E94480A811133
:1045400004C0CF5FC031C1F701C081E0CF910895B1
:104550000E944E0A0C9439181F920F920FB60F92B8
:1045600011248F939F93AF93BF9380917303909186
:104570007403A0917503B09176034196A11DB11DFE
:104580008093730390937403A0937503B0937603A1
:10459000BF91AF919F918F910F900FBE0F901F9081
:1045A000189582E084BD93E095BD9AEF97BD809306
:1045B0006E0008952FB7F89480917303909174035F
:1045C000A0917503B09176032FBF08952FB7F8948B
:1045D00060917303709174038091750390917603D9
:1045E0002FBF0895CF92DF92EF92FF920F931F9308
:1045F0002FB7F89440917303509174036091750341
:10460000709176032FBF6A017B01EE24FF248C0199
:1046100020E030E0C016D106E206F30610F4415067
:1046200051099A01281B390BC9011F910F91FF9065
:10463000EF90DF90CF9008951F920F920FB60F92D8
:1046400011248F939F93AF93BF93809173039091A5
:104650007403A0917503B09176030196A11DB11D5D
:104660008093730390937403A0937503B0937603C0
:10467000BF91AF919F918F910F900FBE0F901F90A0
:1046800018950E948414F89487E797E7909301089F
:104690008093000887E090EBDC0180938503909382
:1046A0008603A0938703B09388039CE088E10FB64C
:1046B000F894A895809360000FBE90936000FFCFA0
:1046C00080E090E008950895CF93C82F1F928F93B4
:1046D00082E897E09F938F930E943F0681E090E0ED
:1046E000A0E0B0E0BC01CD0104C0660F771F881FB9
:1046F000991FCA95D2F70E94BA1F0F900F900F9082
:104700000F90CF910C943918CF938732A8F58E3142
:1047100008F02BC1803109F49FC0F8F4873009F408
:1047200064C0A8F4863009F024C180917203817FAF
:104730008E7F8093720387E897E00E94A6058AE641
:104740009AE00E94A60581E0809377034CC08B30ED
:10475000F1F18E3009F46CC00CC1863109F4B0C09F
:1047600020F4813109F4EDC004C1893109F491C00C
:104770008B3109F449C0FDC0883349F150F48932C6
:1047800009F4F1C0853309F4EEC0873209F0F1C0B5
:10479000EAC0833409F4E7C028F48A3308F4E9C096
:1047A0008953E4C0883409F0E4C00E94391889E5CF
:1047B0009AE00E94A6052FEF83ED90E32150804000
:1047C0009040E1F700C000000E9441230CC082EA43
:1047D00097E05CC080E49AE00E94A6058091720395
:1047E000816080937203C1E0C9C080917203C82FB9
:1047F000C17080FFEFCF8CE49AE00E94A605809103
:104800007203817F8E7F3DC09091720391FBCC2714
:10481000C0F981E0C827892FC0FB81F9809372031A
:10482000CC2319F083E39AE027C085E29AE02EC0FA
:104830009091720392FBCC27C0F981E0C827892FA1
:10484000C0FB82F980937203CC2319F086E19AE0D1
:1048500013C086E09AE01AC09091720393FBCC27B4
:10486000C0F981E0C827892FC0FB83F980937203C8
:10487000CC2351F08AEF99E00E94A6058091720343
:104880008160809372037AC08DEE99E00E94A60544
:10489000AACF8EED99E00E94A60588EB99E00E94D0
:1048A000A60580E799E00E94A60588E499E00E94A9
:1048B000A6058CEF98E00E94A60580ED98E0E6CF73
:1048C00082EC98E00E94A6050E94B1151F928F937A
:1048D00088EA98E09F938F930E943F06809114018D
:1048E0001F928F9381E998E09F938F930E943F06D8
:1048F000809177021F928F938EE798E09F938F931A
:104900000E943F06809115011F928F938BE698E0DD
:104910009F938F930E943F060E94E6229F938F935E
:104920007F936F9384E598E09F938F930E943F0657
:104930008DB79EB746960FB6F8949EBF0FBE8DBF3B
:1049400052CF0E943918C091150181E0C827C09349
:104950001501CC2329F08AE498E00E94A6050EC038
:104960008FE398E093CF80E001C08D510E946423D3
:104970003ACF8DE398E00E94A605C0E08C2FCF913E
:10498000089580E008950C94C124CF93C82F80919E
:104990007703882319F0813059F042C0E091160165
:1049A000F09117018081823261F08434D9F509C019
:1049B000E0911601F09117018081823211F0843468
:1049C00061F48C2F0E94C324811104C08C2F0E949B
:1049D000842324C081E090E021C08C2F0E94C12458
:1049E00081111BC0C43189F018F4CB3029F010C0FC
:1049F000C93259F0C83361F487E897E00E94A605F0
:104A00008EE797E00E94A60508C0109277030CC0BD
:104A10008CE797E00E94A60507C081E0817006C080
:104A20001092770380E002C080E0F8CFCF91089524
:104A30000024552704C0080E591F880F991F00979E
:104A400029F076956795B8F37105B9F7802D952F04
:104A50000895EE0FFF1F0590F491E02D0994F8944E
:024A6000FFCF86
:104A62000080FFFF0556010000FFB80D250EBB0DAB
:104A7200F00DBC0D0101500340362239A806720622
:104A820050061706A305BC05D505F505000008006C
:044A9200040002001A
:106800008800EA44E944E244040005000600070069
:10681000080009000A000B000C000D000E000F001C
:1068200010001100120013001400150016001700CC
:10683000180019001A001B001C001D001E001F007C
:10684000200021002200230024002500260027002C
:10685000280029002A002B002C002D002E002F00DC
:10686000300031003200330034003500360037008C
:10687000380039003A003B003C003D003E003F003C
:1068800040004100420043004400450046004700EC
:10689000480049004A004B004C004D004E004F009C
:1068A000500051005200530054005500560057004C
:1068B000580059005A005B005C005D005E005F00FC
:1068C0006000610062006300640065A185006700EC
:1068D000680069006A006B006C006D006E006F005C
:1068E0007000710072007300890087008A008B00BD
:1068F000E000E100E200E300E400E500E600E7007C
:106900000100010001000100EA4401000100E2442D
:106910000100010001000100460001004A004B0097
:10692000010001004700480001000100E9440100A6
:106930000100010001000100010001003A003B00DC
:106940003C003D003E003F0040004100420043004B
:10695000010035004C0039000100440045005200A0
:1069600049000100010050004F0029004D004E0079
:1069700051000100010001000100010001000100BF
:1069800001000100010001000100010001000100FF
:1069900001000100010001000100010001004D00A3
:1069A0004A004E004B0001000100010001000100FF
:1069B00001000100010001000100010001000100CF
:1069C00001000100010001000100010001000100BF
:1069D00001000100010001000100010001000100AF
:1069E0000100010001000100490001000100010057
:1069F000010001000100010001000100010001008F
:00000001FF
